S020000062696E2F64656D6F70726F675F656B5F6C6D3373363936352E7372656358
S11380008C0B00209992000025930000259300001A
S1138010259300002593000025930000259300007C
S1138020259300002593000025930000259300006C
S1138030259300002593000025930000E19500009E
S1138040259300002593000025930000259300004C
S1138050259300002593000025930000259300003C
S1138060259300002593000025930000259300002C
S1138070259300002593000025930000259300001C
S1138080259300002593000025930000259300000C
S113809025930000259300002593000025930000FC
S11380A025930000259300002593000025930000EC
S11380B025930000259300002593000025930000DC
S11380C025930000259300002593000025930000CC
S11380D025930000259300002593000025930000BC
S11380E025930000259300002593000025930000AC
S11380F0EE11AA5510B5054C237833B9044B13B1CE
S11381000448AFF300800123237010BD0800002051
S11381100000000024A70000084B10B51BB108495B
S11381200848AFF300800848036803B910BD074B43
S1138130002BFBD0BDE81040184700BF0000000032
S11381400C00002024A7000008000020000000000C
S1138150024A136843F005031360704710E000E01F
S1138160024A136843F002031360704710E000E012
S113817010B5441EB4F1807F03D3D021024801F02E
S1138180CBF8024B1C6010BD14A6000014E000E004
S113819038B50C46054620B940F26B21114801F070
S11381A0BBF824B94FF41B710E4801F0B5F80E4B1F
S11381B01B6813F0E04F0ED00B4B1A680B4B1340A7
S11381C0B3F1805F0AD00A4B1B682B60094B1B6814
S11381D02360002038BD4FF0FF3038BD4FF0FF3032
S11381E038BD00BF2CA6000000E00F400000FF7067
S11381F0E0E10F40E4E10F40B0F1402F44D0344BB4
S1138200984243D0A3F5A623984241D003F5A8236E
S113821098423FD0A3F5A62398423DD003F5A82366
S113822098423BD0A3F5A623984239D003F5A8235E
S1138230984237D0A3F55C33984235D003F56033C8
S1138240984233D0A3F55C33984231D003F56033C0
S113825098422FD0A3F55C3398422DD003F56033B8
S113826098422BD0A3F55C33984229D003F56033B0
S1138270984227D0A3F50833984225D003F50C3350
S1138280984223D101207047012070470120704794
S1138290012070470120704701207047012070477A
S11382A0012070470120704701207047012070476A
S11382B0012070470120704701207047012070475A
S11382C0012070470120704701207047002070474B
S11382D00080054070B505460C461646FFF78CFF36
S11382E018B9E421124801F017F8022E03D9E62147
S11382F00F4801F011F805F5806316F0010F03D063
S1138300D5F80024224303E0D5F8002422EA04022D
S11383101A6005F5846316F0020F03D0D5F8202403
S1138320144303E0D5F8202422EA04041C6070BD41
S113833044A60000F8B504460D4617461E46FFF74E
S11383405BFF20B94FF4DD714E4800F0E5FF7B1E62
S1138350012B08D9042F06D00C2F04D04FF4DF7161
S1138360484800F0D9FF082E0FD00A2E0DD00C2E4D
S11383700BD0092E09D00B2E07D00D2E05D026B117
S113838040F2C5113F4800F0C7FF04F5A06317F0A1
S1138390010F03D0D4F800252A4303E0D4F80025C4
S11383A022EA05021A6004F2045317F0020F03D004
S11383B0D4F804252A4303E0D4F8042522EA05026C
S11383C01A6004F5A16317F0040F03D0D4F808254C
S11383D02A4303E0D4F8082522EA05021A6004F5CA
S11383E0A36317F0080F03D0D4F818252A4303E039
S11383F0D4F8182522EA05021A6004F20C5316F088
S1138400010F03D0D4F80C252A4303E0D4F80C253B
S113841022EA05021A6004F5A26316F0020F03D0E3
S1138420D4F810252A4303E0D4F8102522EA0502E3
S11384301A6004F2145316F0040F03D0D4F8142570
S11384402A4303E0D4F8142522EA05021A6004F250
S11384501C5316F0080F03D0D4F81C252A4303E05C
S1138460D4F81C2522EA05021A6004F5A5631EB996
S1138470D4F82825154303E0D4F8282522EA050575
S11384801D60F8BD44A6000070B504460D461646AE
S1138490FFF7B2FE20B94FF45171034800F03CFFDE
S11384A044F8256070BD00BF44A6000038B50446FA
S11384B00D46FFF7A1FE20B940F20441074800F041
S11384C02BFF012229462046FFF704FF082301223F
S11384D029462046FFF72EFF38BD00BF44A6000002
S11384E038B504460D46FFF787FE20B940F21F5108
S11384F0074800F011FF022229462046FFF7EAFE52
S11385000823012229462046FFF714FF38BD00BF87
S113851044A6000038B504460D46FFF76DFE20B9A9
S113852040F2C651074800F0F7FE022229462046D1
S1138530FFF7D0FE0823042229462046FFF7FAFE5F
S113854038BD00BF44A60000F0B5864600F1100512
S113855003699FB2C3F3074008701B0E4B70B81F2A
S113856006469042A8BF1646022302E02C68CC506F
S11385700433341FA342F9DDB34223DADEF810409A
S1138580A6F1030E73450BD103F1010ECC549E1CCE
S11385904FEA142C01F80EC0240C8C55043311E05E
S11385A0A6F1020E734505D15E1CCC54240A8C55E9
S11385B0043307E0013EB34204D1CC54043301E058
S11385C029680433B91E8B42FADB904200DD404235
S11385D0F0BD00BF40F2FE739A4201DD5042704785
S11385E030B4A2F10E030C7843EA04434C7843EA16
S11385F0046300F110050361022302E0CC582C60EF
S11386000433141FA342F9DD93421CD0D41EA342A9
S11386100AD15D1CCC5C02334D5D44EA0524CB5C7D
S113862044EA034303610EE0941EA34206D15C1C9A
S1138630CB5C095D43EA0123036104E0541EA342B9
S113864001D1CB5C036101238363104630BC7047C6
S113865038B505460C46074B984203D04E210648D0
S113866000F05AFE054BA3FB0434C4F347546C6278
S113867038BD00BF008004405CA600006BCA5F6B7D
S113868038B505460C46124B984203D09521114843
S113869000F042FE24F4873323F016031BB1992122
S11386A00C4800F039FEEB6823F01602E3B21343E2
S11386B0EB60AB6823F00E02C4F307231343AB60F3
S11386C0EB6B23F00103C4F307441C43EC6338BD94
S11386D0008004405CA6000030B583B005460C461B
S11386E0134B984204D04FF48171124800F014FEE9
S11386F024B940F203110F4800F00EFE23788DF8E0
S1138700043063788DF80530A3788DF80630E3786B
S11387108DF80730019B6B610023019323798DF859
S1138720043063798DF80530019BAB6103B030BD33
S1138730008004405CA6000010B504460C4B98422F
S113874004D04FF4AC710B4800F0E6FDA36843F08D
S11387501003A360A36843F00103A360E36843F03C
S11387600103E360A36843F01003A36010BD00BFDE
S1138770008004405CA6000070B504460D46164611
S1138780104B984204D040F27F210F4800F0C4FD02
S113879025B94FF420710C4800F0BEFD002E04DC16
S11387A040F28121084800F0B7FD636B13F03F0FDE
S11387B005D0324629462046FFF7C6FE70BD00208C
S11387C070BD00BF008004405CA6000070B5044684
S11387D00D4616460F4B984204D040F28E310E4897
S11387E000F09AFD25B940F28F310B4800F094FD5A
S11387F0002E04DC4FF46471074800F08DFDA36B78
S113880013F0010FFBD1324629462046FFF7E2FE62
S113881070BD00BF008004405CA6000038B504466B
S11388200D460A4B984204D040F23541084800F006
S113883073FD35F07F0304D04FF48761044800F0E2
S11388406BFD616821EA0501616038BD0080044068
S11388505CA6000038B504460D46064B984204D089
S11388604FF48B61044800F057FD20680DB1636834
S1138870184038BD008004405CA6000038B50446AA
S11388800D46094B984204D040F28D41074800F050
S113889043FD35F07F0304D04FF49261034800F0A8
S11388A03BFD256038BD00BF008004405CA600008D
S11388B038B504460D460D4B984204D040F2DC41D5
S11388C00B4800F029FD04F12003226A12F0010F85
S11388D0F9D1ED00EDB245F001051D601A6812F002
S11388E0010FFBD1206B80B238BD00BF0080044073
S11388F05CA60000094B984209D003F580539842C6
S113890007D003F58053984205D101207047012018
S11389107047012070470020704700BF00C000402E
S113892010B50446FFF7E6FF20B94FF4CF710748AE
S113893000F0F2FCE36A43F01003E362236B43F4B8
S1138940407343F00103236310BD00BF78A6000009
S113895010B50446FFF7CEFF20B94FF4DF71094884
S113896000F0DAFCA36913F0080FFBD1E36A23F0EB
S11389701003E362236B23F4407323F001032363A6
S113898010BD00BF78A60000F8B505460C46164693
S11389901F46FFF7AFFF20B940F20D112F4800F03A
S11389A0BBFC26B94FF487712C4800F0B5FC2C4B66
S11389B01B6813F0E04F1FD0294B1A68294B134052
S11389C0B3F1805F1AD0264B1A68264B1340264A0F
S11389D0934204D1224B1B689BB2022B10D0204B34
S11389E01A68204B1340214A93420BD11C4B1B683D
S11389F09BB24BB1082308E0102306E0102304E0E7
S1138A00102302E0082300E0102306FB03F3A34233
S1138A1004D940F20F11114800F07EFC2846FFF7FC
S1138A2097FFB4EB061F05D22B6B43F020032B6397
S1138A30760803E02B6B23F020032B63E400B4FBE4
S1138A40F6F40134E3096B62C4F34504AC62EF62EB
S1138A500023AB612846FFF763FFF8BD78A600004A
S1138A6000E00F400000FF70000001100000031040
S1138A7010B50446FFF73EFF20B940F2094106480D
S1138A8000F04AFCA36913F0100F01D1206810BD57
S1138A904FF0FF3010BD00BF78A60000A0F5801392
S1138AA0013B012B40F28F80714B984200F08D8086
S1138AB003F58073984200F08A8003F500739842AE
S1138AC000F0878003F18053A3F54073984200F0CF
S1138AD0828003F5807398427FD003F50073984237
S1138AE07DD003F5705398427BD003F11023984254
S1138AF079D0604B984278D00133984277D00233D2
S1138B00984276D00433984275D00833984274D092
S1138B101033984273D02033984272D04033984235
S1138B2071D08033984270D0402870D0B0F1102FAB
S1138B306FD0514B98426ED003F57D2398426CD090
S1138B4003F18053A3F57063984268D04B4B98426D
S1138B5067D0703B984266D0B0F1101F65D0484B87
S1138B60984264D003F58073984262D0A3F5F873F9
S1138B70984260D0103398425FD003F1005398427A
S1138B805DD0404B98425CD0013398425BD00233B5
S1138B9098425AD00433984259D03B4B984258D00B
S1138BA00133984257D00233984256D0B0F1202F67
S1138BB055D0364B984254D0082854D0344B984260
S1138BC053D10120704701207047012070470120D4
S1138BD07047012070470120704701207047012031
S1138BE07047012070470120704701207047012021
S1138BF07047012070470120704701207047012011
S1138C007047012070470120704701207047012000
S1138C1070470120704701207047012070470120F0
S1138C2070470120704701207047012070470120E0
S1138C3070470120704701207047012070470120D0
S1138C4070470120704701207047012070470120C0
S1138C5070470120704701207047012070470120B0
S1138C60704701207047012070470020704700BF03
S1138C7000011000010000200040001080000030BE
S1138C80000100100100101001000010010010206C
S1138C900010100010B582B00446FFF7FFFE20B9A3
S1138CA040F2B9110F4800F037FB220F0E4B53F876
S1138CB022201168A3B2C4F3044403FA04F441EA81
S1138CC0040313600023019302E0019B0133019329
S1138CD0019B0F2BF9D9136823EA0404146002B032
S1138CE010BD00BFECA6000010A7000010B504469C
S1138CF0FFF7D4FE20B94FF4FC71084800F00CFBD8
S1138D00220F074B53F822100868A2B2C4F304439D
S1138D1002FA03F303430B6010BD00BFECA600008E
S1138D2004A70000014A024B1A60FEE70400FA059A
S1138D300CED00E001387FF4FDAF704770B54E4B89
S1138D401B6813F0E04F06D04B4B1A684B4B134093
S1138D50B3F1805F02D10028C0F28C8004464849F8
S1138D600B68484A166823F4800545F4006546F408
S1138D7000600D60106013F0020F02D014F0020FB7
S1138D8005D013F0010F1ED014F0010F1BD164F0B5
S1138D9003031D403A4B1D60002805DA06F07003FA
S1138DA0302B07D0702B05D0002808DB05F03003EA
S1138DB0302B04D14FF48050FFF7BCFF03E04FF495
S1138DC00020FFF7B7FF25F45F5525F0300543F287
S1138DD0F07323401D432C4B334043F400622B4B70
S1138DE023401343E20002F0400240202849086077
S1138DF053EA020604D5234B1E60103B1D6003E0BA
S1138E001F4B1D6010331E601020FFF793FF25F0E9
S1138E10F86525F003051F4A2240154326F0FC514E
S1138E2004F0FC530B4314F0804F07D045F4800545
S1138E3023F4800318492140194301E023F08041C1
S1138E4014F4006F07D00EE0144A126812F0400FB9
S1138E5005D1013B01E04FF40043002BF4D125F48C
S1138E60006521F40061064B1D6010331960102069
S1138E70FFF760FF70BD00BF00E00F400000FF700F
S1138E8060E00F4070E00F408FDFFF7F30200080F4
S1138E9058E00F400300C0070000404050E00F407E
S1138EA030B4724B1B68724A1168002902DA01F06F
S1138EB0700201E003F03002202A3AD003D862B1F4
S1138EC0102A10D0CFE0602A5BD0702A56D0302A06
S1138ED040F0C98047F2305069E0C3F3841265481A
S1138EE050F8220063E0644A126812F0E04F4BD05D
S1138EF0614A1068614A0240B2F1805F46D05E4A1E
S1138F0010685E4A02405E48824204D15A4A12689E
S1138F1092B2022A3CD0584A1068584A0240594832
S1138F20824237D1544A126892B2002A34D0564849
S1138F303DE0514A126812F0E04F2FD04E4A1068BB
S1138F404E4A0240B2F1805F2AD04B4A10684B4A25
S1138F5002404B48824204D1474A126892B2022A24
S1138F6020D0454A1068454A0240464882421BD1F7
S1138F70414A126892B2CAB1444818E04FF4004022
S1138F8015E04FF4800012E0414810E040480EE044
S1138F9040480CE03C480AE03E4808E03E4806E011
S1138FA03D4804E03D4802E0384800E03B480029E1
S1138FB002DA11F4006F04D000292FDB13F4006FE0
S1138FC02CD1374A1468643A126812F0E04F06D084
S1138FD0294A1568294A2A40B2F1805F0AD1C4F3AC
S1138FE04812023202FB00F004F01F020232B0FB0E
S1138FF0F2F009E0C4F3481202FB00F004F01F028F
S113900001325200B0FBF2F014F4804F00D040085B
S113901014F4004F00D0800843F4800313F4800F4D
S113902022D0002919DA11F0804F10D0002902DA79
S113903011F4006F04D0002909DB13F4006F06D18A
S11390404000C1F386530133B0FBF3F00CE0C1F3ED
S1139050C5530133B0FBF3F006E0C3F3C35301334C
S1139060B0FBF3F000E0002030BC704760E00F403C
S113907070E00F4090A6000000E00F400000FF7079
S113908000000110000003100024F40000093D005A
S1139090C0E1E400001BB70070383900C0C62D00E1
S11390A064E00F4010B5044C2046FFF71FFE204635
S11390B0FFF7F0FD10BD00BF0050102030B585B0A3
S11390C03F48FFF713FE0C213E48FFF723FA3E4CBE
S11390D07F212046FFF7A2FB00212046FFF7BAFBC1
S11390E001462046FFF7CAFBFFF7DAFE0146204699
S11390F0FFF7AEFA16212046FFF7C2FA2046FFF723
S11391001BFB01212046FFF7D3FB044600F062FA63
S113911000F59C55083508E001212B48FFF7C8FBF2
S1139120044600F057FA854202D914F0040FF3D034
S113913008238DF8083000238DF8093027238DF893
S11391400A3069238DF80B305B238DF80C304523EE
S11391508DF80D30694601A8FFF71AF8019BB3F1A9
S1139160FF3F13D0009AB2F1FF3F0FD08DF80830C3
S1139170190A8DF809101B0C8DF80A308DF80B2094
S1139180130A8DF80C30120C8DF80D2002A90E482C
S1139190FFF7A2FA9DF808200C4B1A709DF80920DD
S11391A05A709DF80A209A709DF80B20DA709DF889
S11391B00C201A719DF80D205A7105B030BD00BF06
S11391C02000002000500240008004409000002055
S11391D038B50B4D00212846FFF73CFB04460146F9
S11391E02846FFF74BFB14F0010F06D040F2426211
S11391F004492846FFF7C0FA38BD002038BD00BF37
S1139200008004404801002008B5034B1A88034934
S11392100348FFF7DBFA08BD0001002048010020E5
S11392200080044010B50748FFF760FD064C01219B
S11392302046FFF73BF9002201212046FFF724F9DD
S113924010BD00BF200000200050024010B500F007
S1139250C1F90E4B1B68C31AB3F5FA7F14D3044645
S11392600B4B1B783BB90121094B19700A4609487D
S1139270FFF70AF906E00022054B1A7001210548A0
S1139280FFF702F9014B1C6010BD00BF2400002051
S1139290280000200050024008B50F498D460B4BB2
S11392A00B4A03E0116819600433043209498B4204
S11392B0F8D30A480A494FF000028842B8BF40F880
S11392C0042BFADB00F01AF808BD00BF00000020F0
S11392D028A70000080000208C0B002008000020B4
S11392E08C07002008B50448FFF728FDFFF79AFF14
S11392F000F05CF908BD00BF8003C00108B5FFF7AA
S1139300F1FF00F093F800F03BF8FFF79FFF00F047
S1139310DBF800F087F8F8E7014B1960FEE700BFBF
S11393202C000020FEE700BF08B50A48FFF7DEFC6A
S11393300948FFF7DBFC03214FF04020FFF7D0F88A
S1139340FFF7AEFD60234FF4614201460348FFF787
S11393501BFB08BD010000100100002000C00040FC
S113936010B504460548FFF783FBB0F1FF3F02D078
S11393702070012010BD002010BD00BF00C00040BF
S113938008B5FFF7D1FF08BD08B5FFF7CBFC08BD52
S113939008B5204B1B789BB91F48FFF7E1FF012854
S11393A037D11D4B1B78002B33D000F013F91B4B26
S11393B018600122174B1A700022194B1A7008BD4D
S11393C0174B1B78013314481844FFF7C9FF0128D1
S11393D015D1134A13780133DBB213700E4A127895
S11393E0934216D100220B4B1A700B4B5B78FF2B68
S11393F00FD1094B9B7863B9FFF7C6FF08BD00F096
S1139400E9F8064B1B686433984202D90022014BE9
S11394101A7008BD760000203400002030000020BF
S11394207500002008B5FFF7B3FF08BD08B5FFF7C6
S113943039FE00F0CFF800F5FA70124B186000F016
S1139440C9F800F51C5010300F4B186000F034F9C7
S11394500E4B4FF6A9621A8043F6137159800C4BD8
S11394604FF6FF711980002159800A4B1A8040F28F
S113947013125A804EF6030000F04CF9FFF71EFE5B
S113948008BD00BF7C0000207800002044010020BB
S1139490400100203C01002008B5094B1B7813F063
S11394A0400F0BD113F0020F08D0064B1B681A793A
S11394B0FF2A03D15B790BB9FFF766FF08BD00BF34
S11394C00C0100201001002010B5FFF781FE48B305
S11394D02D4A10802D4B9C894FF4006000F034F924
S11394E084420DD1012000F069F9274B1B88CBB1D0
S11394F000F0D4FFFFF788FE0022234B1A8011E00E
S1139500224B9C8940F6060000F01EF9844209D1E2
S113951000F054FF1C4B1B8823B1FFF775FE00229B
S1139520194B1A8000F056F8194B1B6898421CD34B
S113953003F5FA73164A1360002414E0C4EB041311
S11395405A00144B1344144A1360022000F036F9F5
S11395500D4B1B8833B100F0A1FFFFF755FE00222D
S1139560094B1A800134002CE8D000F033F80B4B7F
S11395701B68984206D303F51C531033074A136043
S113958000F0ECFE10BD00BF0001002048010020E7
S11395907C00002018010020140100207800002025
S11395A0014B1860704700BF8000002008B5FFF72A
S11395B077FC074BA3FB00308009FEF7D9FDFEF7CB
S11395C0C7FDFEF7CDFD0020FFF7EAFF08BD00BF91
S11395D0D34D6210014B1868704700BF8000002013
S11395E0024A136801331360704700BF80000020F3
S11395F010B4013A0A440BE00C784B7803EB0423D3
S11396009BB2184480B2834201D9013080B2023146
S11396109142F1D307D10B781B02184480B28342E4
S113962001D9013080B210BC704700BF70B4C57856
S11396300D44EDB2134CE57083780E0A3344DBB26B
S1139640A37042786270007820709CB2A64206D95A
S11396500132D2B20B4C62700AB901302070C9B227
S11396608D420CDA0133DBB2064A93703BB953786E
S11396700133DBB2537013B913780133137070BC28
S1139680704700BF0801002010B5094C236801464B
S113969003F10800FFF7CAFF2368064A117819721C
S11396A05178597291789972D278DA7210BD00BFEC
S11396B014010020080100200022124B1A7006E059
S11396C00021114A22F8131001330E4A13700D4B76
S11396D01B78002BF4D000220A4B1A7009E0C3EB6C
S11396E003114A0009490A44002151760133054A0D
S11396F01370044B1B78002BF1D04FF48062044BA1
S11397001A8070478E0000203801002018010020C4
S11397108C00002000220A4B1A700BE01946094AFB
S113972032F813201AB9074B23F81100704701339C
S1139730034A1370024B1B78002BEFD0704700BF15
S11397408E00002038010020030A43EA002080B282
S1139750704700BF08B5142205490020FFF748FFF1
S113976010B1FFF7F1FF08BD4FF6FF7008BD00BF51
S11397705601002038B50D4D2C7C6B7C03EB042482
S1139780143CA4B22044082205F11A0180B2FFF768
S11397902FFF224605F12201FFF72AFF10B1FFF740
S11397A0D3FF38BD4FF6FF7038BD00BF480100201D
S11397B008B50620FFF7DEFF08BD00BF70B5934B68
S11397C01C68934B934A1360934A136003280FD188
S11397D0637E03F00F03032B40F02F85238A002BB5
S11397E040F02B8508228D4B1A70FFF755FEEAE3F3
S11397F0022879D18A4AD3780133DBB2D37063B9B2
S113980093780133DBB293703BB953780133DBB205
S1139810537013B91378013313700023814A1380F2
S1139820814A1380637E072B01D0052B0AD1A37EC6
S11398300133DBB2A376782B40F0FF8400236376F8
S113984000F0FBBC002B00F0F884228A002A40D0F0
S1139850A27E511EA176002A40F0EF84E27E082AFF
S113986005D0591EC9B201290ED8052A0CD10023EE
S113987063768022694B1A70FFF70EFE14226B4B3D
S113988083F82F2000F05BBC042A03D80321914005
S1139890C9B200E03021A1760132E27603F00F0371
S11398A0013B072B00F2C984DFE813F0BE01080076
S11398B00D003803C7043803C704380300225B4B88
S11398C083F82F20B4E10422544B1A70FFF7E4FD0F
S11398D0AEE303F00F03032B40F0AF8408224F4B99
S11398E01A70FFF7D9FD6EE3504B9B7B452B40F07C
S11398F0A4844E4A157C537C03EB0521494A128803
S1139900914200F39A848DB2464B1D80474B1B7DD8
S113991013F03F0F40F09184444B5B7D002B40F0EB
S11399208C84434B1C880CB95B885BB13F4BDB8B4D
S11399309C4240F082843D4B1A8C3D4B5B889A429A
S113994040F07B84FFF706FF4FF6FF73984240F028
S11399507484364BDB7D062B23D0012B40F06D84C1
S1139960324B93F82230082B40F067842F4B0022AF
S113997083F822209B8C4FF6F672934203D9093365
S11399802A4A938402E00833284A9384274B5A8B4B
S1139990DA839A8B1A845C83254A52889A8300F06E
S11399A048BCFFF705FF4FF6FF73984240F045842B
S11399B0204C17E0617EA1B11C4B9A8CA3889A427B
S11399C00FD11A4B5A8CE3889A420AD1174B5A8BFF
S11399D023889A4205D1154B9A8B63889A4200F0EA
S11399E041811E34134B9C42E4D9104B93F82F3021
S11399F003F03F03022B2FD10C4B9B8C99B20E4AE0
S1139A00138000220D4B1A7022E000BF14010020C5
S1139A107E01002010010020040100200C01002020
S1139A2088000020000100208A070020480100204F
S1139A304401002018010020840000208E00002032
S1139A40924A32F8132091425BD00133904A13704A
S1139A508F4B1B78002BF3D08E4B93F82F3013F0E1
S1139A60040F40F0EA838B4B142283F82F20282123
S1139A70894A1180502283F82E2093F8290093F804
S1139A802D2083F8292093F8281093F82C2083F8AC
S1139A90282083F82C1093F8272093F82B4083F880
S1139AA0274083F82B2093F82640794D2C7093F8A7
S1139AB02A5083F8265083F82A400130C0B283F834
S1139AC02D0068B94B1CDBB2724981F82C303BB9CC
S1139AD0531CDBB281F82B3013B9013481F82A40CE
S1139AE06C4B5A8C6D490A80998C59849A845A8B90
S1139AF0DA839A8B1A846A4A1188598352889A8322
S1139B006FE30024624B1C701CE019461E2265485A
S1139B1002FB0302527E1AB91E2404FB010415E061
S1139B20072A0CD13CB11E225E4902FB0312917E2E
S1139B30A27E914203D95B4A1E2404FB0324013311
S1139B40534A1370524B1B78002BDED0002C00F0CC
S1139B507483554B1C600323A37623760023A375DB
S1139B600422E275E3764B4DAB8CA3806B8CE380CF
S1139B706B8B2380AB8B6380012060764B4B1A7810
S1139B8022735A7862739A78A273DB78E373208223
S1139B9095F82930E37295F82830A37295F82730A8
S1139BA0637295F826302372FFF76EFD95F82E0048
S1139BB000F0F003502B37DD0022354B1A702BE0F8
S1139BC003F13602334DAA5C72B3012A03D1013387
S1139BD02F4A137020E0022A16D103F137022D4DCB
S1139BE0AA5C042A10D101F13803EA5C39316B5CB8
S1139BF043EA0222294B1A8040F20A63934228BFA7
S1139C0013466382A3820FE003F1370221498A5C81
S1139C1052B113441E4A13701D4B1B781946020996
S1139C20053AB3EB820FCBDB10221A4B83F82F20BB
S1139C30184B93F82F2042F0020283F82F200222BF
S1139C4083F83620042283F83720062283F838204C
S1139C500A2283F839202C210F4A1180602283F8CC
S1139C602E2073E2104B1C600022114B1A70094B1A
S1139C7093F82F2012F0040F1CD0002363762022C7
S1139C800B4B1A70FFF708FCD7E200BF3801002025
S1139C908E000020480100200001002084000020E4
S1139CA04401002018010020140100208800002035
S1139CB00C0100209C4B93F82E301B099B009B4801
S1139CC00370EB1A143B9BB29948038001F00F0117
S1139CD0022903D102F03F0112290FD013B912F067
S1139CE0030F0BD0904BD98C2389994240F02382E7
S1139CF08D4B198D6389994240F01D8212F0100F2B
S1139D0047D0218A002944D004F10C00FFF78EFCCF
S1139D10854B93F82A30874A1078834239D1824B95
S1139D2093F82B3051788B4233D17F4B93F82C30FE
S1139D30927893422DD17C4B93F82D507D4BDB7858
S1139D409D4226D120736173A273E373E37ECBB982
S1139D50237EA27E9A1AD2B2A17DA2EBD102D2B204
S1139D6053B21144C9B2A175002B01DA524253B265
S1139D70E07DA3EB9002D2B20244D3B2E37503EBCD
S1139D80D103237601226C4B1A70237EA376002321
S1139D902382617E01F00F03013B072B00F24D8209
S1139DA0DFE813F00800230096007301A201BE014E
S1139DB0C9016501604B1B7813F0010F00F03D826F
S1139DC00323637640225C4B1A7000232382584B92
S1139DD0188820B14222584B1A70FFF755FC002214
S1139DE0564B1A80FFF758FBEDE0534B1B7813F0EA
S1139DF0010F63D04C4B93F82F3003F03F03122B29
S1139E005CD1494B93F82E0000F0F003502B37DD62
S1139E100022464B1A702BE003F13602424DAA5C35
S1139E2072B3012A03D10133404A137020E0022A9D
S1139E3016D103F137023C4DAA5C042A10D101F17A
S1139E403803EA5C39316B5C43EA02223C4B1A80EA
S1139E5040F20A63934228BF13466382A3820FE051
S1139E6003F1370230498A5C52B113442F4A13700C
S1139E702E4B1B7819460209053AB3EB820FCBDB54
S1139E8003236376284B93F82620227293F8272025
S1139E90627293F82820A27293F82930E3720120A9
S1139EA0FFF7F2FB4222244B1A7000232382204A3C
S1139EB01380224A1380FFF7EFFA84E020221E4B1E
S1139EC01A70FFF7E9FA1F4B1B6800225A76C3E5A4
S1139ED0154B93F82F3013F0010F35D011F0100FFC
S1139EE032D1238A002B40F0A881114D28880130FB
S1139EF080B2FFF7C9FB104A137843F010031370C4
S1139F002A881AB143F002030B4A1370FFF7C4FA0C
S1139F1001232382082363760023E3761122024B74
S1139F2083F82F200BE100BF480100208E000020A1
S1139F3000010020080100200C0100208A070020F5
S1139F40840000201401002013F0200F10D0994841
S1139F5090F834301A0290F8353043EA0200964DF6
S1139F602E6830442860954813430288D31A03802E
S1139F70924B188848B111F0100F06D1904A13780B
S1139F8043F002031370FFF77FFB8A4A92F8301004
S1139F9092F8313003EB01239BB28A4A1380A28AE0
S1139FA0934200D80BB9874B1A80864B1B88638277
S1139FB0834B1B7813F0030F00F03F810022824B88
S1139FC01A80FFF769FA7E4B1B7813F0200F08D034
S1139FD000237D4A138063761422764B83F82F2066
S1139FE0ADE013F0100F0CD00023774A1380012248
S1139FF0228204226276E37611226E4B83F82F20AC
S113A0009DE0714A12888AB113F0010F01D0002338
S113A0102382238A43B9638A9A4201D96A4A138004
S113A020694B1B88238201E0674A13800023E3768F
S113A030664B1A68604B1A60634B1B884BB1238ACA
S113A0403BB128335D4A138018225A4B83F82F20E2
S113A05078E05B4B1B7813F0020F00F0EE802822AF
S113A060564B1A801022534B83F82F206AE0544B2E
S113A0701B7813F0010F00F0E080002363761022B8
S113A0804F4B1A70FFF708FAD7E04C4B188808B109
S113A090FFF7FAFA474B93F82F3013F0010F15D05E
S113A0A0474B1B7813F0010F05D007236376002379
S113A0B0A376238201E0062363760120FFF7E4FA06
S113A0C010223F4B1A70FFF7E7F934E03C4B1B7842
S113A0D013F0010F04D00523637600232382ACE040
S113A0E0364B1B883BBBA8E0344B188808B1FFF7FC
S113A0F0CBFA304B93F82F3013F0010F0CD0072319
S113A10063760023A3760120FFF7BEFA10222C4BBE
S113A1101A70FFF7C1F90EE0284B1B885BB98CE07D
S113A120274B1B7813F0010F00F087800723637619
S113A1300023A37681E010221E4B83F82F202822CF
S113A1401E4B1A8050221B4B83F82E20227A194B67
S113A15083F82A20627A83F82B20A27A83F82C20B1
S113A160E27A83F82D20227B83F82620627B83F811
S113A1702720A27B83F82820E27B83F8292006226B
S113A180DA75A2885A84E2889A84114A118859831C
S113A19052889A832288DA8362881A84637E13F051
S113A1A0100F17D0034B002283F8312083F830209E
S113A1B017E000BF4801002010010020000100202A
S113A1C00C010020840000208A07002004010020E4
S113A1D0440100201C4B062283F830200A2283F815
S113A1E03120194C4023A375184B1B881A0A22747A
S113A1F06374002584F8355084F8345084F8325060
S113A20084F83350FFF7D4FAC04360864523A37320
S113A210E573657525750E4A138801339BB2138067
S113A2201A0AA274E37425766576FFF793FAC0439D
S113A23020830022074B1A7070BD0023034A138049
S113A240044A137070BD00BF4801002000010020C3
S113A250860000200C010020F0B400223A4B1A7052
S113A2601EE03A4D5A001A4494002E192C5BA4B1F6
S113A27003EB4305AA00354D2A4452886AB1058888
S113A280AC420AD14488A24207D10C687460898820
S113A29031812F4A1278B27254E001332A4A137082
S113A2A0294B1B78072BDCD90022274B1A700FE0AF
S113A2B0264D5A001A4494002E192A5B2AB903EB3E
S113A2C04304A2002A44528832B101331E4A137057
S113A2D01D4B1B78072BEBD9082B28D100231D4AD3
S113A2E013701D4A1370184A137013E0184A147837
S113A2F003EB4305AA00154D2A44927AA61A154D7C
S113A3002D78AE4203DD134A1670134A13700133DD
S113A3100D4A13700C4B1B78072BE7D90E4B1B7897
S113A320094A137003EB43039A00084E164402686B
S113A330334643F8042B0A6872608A889A80044B77
S113A3401B78B372F0BC7047960000209800002080
S113A350F900002097000020F800002010B4144BEE
S113A3601C780134E4B21C700022124B1A7019E0FC
S113A37011485A001A4491004218415A52880A431B
S113A3800DD003EB43018A000244927AA21A772A81
S113A39005DD03EB43018A0000200749885001339F
S113A3A0044A1370034B1B78072BE1D910BC704788
S113A3B0F9000020960000209800002010B5324BD0
S113A3C01B88292B03D800222F4B1A8010BD002292
S113A3D02D4B1A802D4B9B8AB3F5807F03D0B3F5A8
S113A3E0007F3FD010BD294BDA8C294B1B889A4241
S113A3F049D1264B1A8D264B5B889A4243D1254C72
S113A4002146A01DFFF728FF002204F8022C022297
S113A41004F8012C2168C4F80A10A188E1811E49BE
S113A420086820608988A18044F8100C24F80C1C6A
S113A430D4F80A1044F8161CE28924F8122CE28895
S113A440228222896282124A1188E1805288228102
S113A450082204F80A2C062204F8092C2A220A4BA2
S113A4601A8010BD094BDA8C094B1B889A420AD119
S113A470064B1A8D064B5B889A4204D10548014667
S113A4800630FFF7E9FE10BD00010020480100205E
S113A490440100205E0100209000002030B44C4BA9
S113A4A0D98B8AB24FF6FF739A420CD1484B188C61
S113A4B04FF6FF73984206D1454B464A1068186020
S113A4C092889A8072E0444B1B8844480088534029
S113A4D0184209D13E4B1A8C94B23F4B5B883F48DB
S113A4E040886340184206D03D4B3E4A118819808B
S113A4F052885A8002E03A4B19805A8000223A4B23
S113A5001A7016E039485A001A4491004518344A22
S113A5101488425A944209D1314A508803EB4301CA
S113A5208A0032490A445288904206D001332E4AA6
S113A53013702D4B1B78072BE4D9082B30D1244BF7
S113A5404FF0FF321A609A8000221A629A842849D6
S113A5500868C3F8060089885981C3F8160059832E
S113A5601F490888D884498819851B490888988315
S113A5704988D9831A75012159759A73D9730821A9
S113A58019745A7406229A740422DA74197306220E
S113A5905A733633174A13602A22174B1A8014E071
S113A5A00B4B55F8042F1A60AA889A80084B104A5E
S113A5B01168C3F8061092885A8108221A7300227F
S113A5C05A730D4A13880E33138030BC704700BF92
S113A5D0480100201CA70000440100204001002085
S113A5E0FC0000203C010020960000209800002080
S113A5F0900000201001002000010020F8B500BFE9
S113A600F8BC08BC9E467047F8B500BFF8BC08BC4F
S113A6109E4670476C69622F6472697665726C69D4
S113A620622F7379737469636B2E63006C69622F94
S113A6306472697665726C69622F666C6173682EE8
S113A640630000006C69622F6472697665726C69DC
S113A650622F6770696F2E63000000006C69622FBF
S113A6606472697665726C69622F65746865726E6E
S113A67065742E63000000006C69622F6472697651
S113A68065726C69622F756172742E63000000003C
S113A69040420F0000201C0080841E000080250022
S113A6A0999E36000040380000093D0000803E00BD
S113A6B000004B00404B4C0000204E00808D5B009E
S113A6C000C05D000080700000127A0000007D0070
S113A6D080969800001BB7000080BB00C0E8CE0045
S113A6E0647ADA000024F4000000FA006C69622F36
S113A6F06472697665726C69622F73797363746CC2
S113A7002E63000000E10F4004E10F4008E10F4018
S113A71040E00F4044E00F4048E00F40FFFFFFFFE0
S10BA720FFFF0000000000002F
S10BA72819810000F580000016
S90380007C
